:1000000012C0C9C02BC02AC029C028C027C026C022
:10001000A8C02EC123C022C021C020C01FC01EC046
:100020001DC01CC01BC011241FBECFE5D4E0DEBF25
:10003000CDBF10E0A0E6B0E0E6E6F3E002C0059038
:100040000D92A236B107D9F710E0A2E6B0E001C0E8
:100050001D92AA36B107E1F71BD183C1D1CFDF933F
:10006000CF93CDB7DEB787E390E02FEFFC0120837D
:1000700088E390E0FC01108284E390E02FEFFC0124
:10008000208385E390E0FC01108281E390E020E38F
:10009000FC01208382E390E0FC011082CF91DF918C
:1000A0000895DF93CF93CDB7DEB782E390E022E3EC
:1000B00030E0F90120812061FC012083CF91DF91A4
:1000C0000895DF93CF93CDB7DEB782E390E022E3CC
:1000D00030E0F90120812F7EFC012083CF91DF9158
:1000E0000895DF93CF93CDB7DEB785E390E025E3A6
:1000F00030E0F90120812062FC012083CF91DF9163
:100100000895DF93CF93CDB7DEB785E390E025E385
:1001100030E0F90120812F7DFC012083CF91DF9118
:100120000895DF93CF93CDB7DEB785E390E025E365
:1001300030E0F90120812860FC012083CF91DF911C
:100140000895DF93CF93CDB7DEB785E390E025E345
:1001500030E0F9012081277FFC012083CF91DF91DE
:1001600008951F920F920FB60F9211248F939F93B1
:10017000DF93CF93CDB7DEB780EA9FE09093640022
:1001800080936300CF91DF919F918F910F900FBE6D
:100190000F901F9018951F920F920FB60F92112477
:1001A0002F938F939F93EF93FF93DF93CF9300D081
:1001B000CDB7DEB780E390E0FC018081882F90E02E
:1001C00084709070009759F08CE490E0FC011182EB
:1001D00010828EE490E021E0FC0120833BC080E3AC
:1001E00090E0FC018081882F90E0847090700097EF
:1001F00089F58EE490E0FC0110828CE490E0FC0133
:10020000808191819A83898389819A81FDE78130F8
:100210009F0738F088EE93E090936400809363002A
:1002200019C089819A812EE38038920728F41092B0
:100230006400109263000EC089819A8180589E43A9
:10024000929582958F7089279F708927909364007B
:10025000809363000F900F90CF91DF91FF91EF910A
:100260009F918F912F910F900FBE0F901F90189517
:100270001F920F920FB60F921124DF93CF93CDB739
:10028000DEB7CF91DF910F900FBE0F901F901895A2
:10029000DF93CF93CDB7DEB7E2DE85E590E021E0D6
:1002A000FC0120838BE590E020E4FC0120838FE4B7
:1002B00090E0FC01108289E590E029E530E0F90149
:1002C00020812460FC0120838EE490E0FC011082F8
:1002D0008CE490E0FC011182108283E590E021E043
:1002E000FC01208389E590E029E530E0F9012081D7
:1002F0002160FC01208378948EE490E021E0FC01F1
:100300002083DFDEFEDE1DDF01C000008091630080
:1003100090916400F3E085389F0710F002DF01C080
:1003200010DF809163009091640021E0813E92078C
:1003300010F0D7DE01C0E5DE80916300909164008B
:10034000893C910510F0ADDE01C0BBDE80916300F9
:1003500090916400893C9105C0F6B3DED2DEF1DEF7
:06036000D5CFF894FFCF99
:02036600010094
:00000001FF
